:100000000AC018951895189518951895189518956B
:100010001895189518958FE181BD87E181BD8FED09
:100020008DBFC0ECE8EB4E2EDD275D2EEEE7F0E055
:10003000A0E6B0E088278D933197E9F76624BC9A53
:10004000C498E1E0F0E00BD0C498E1E0F0E007D024
:10005000C49AE1E0F0E003D0F7CFF894FFCF88EE48
:1000600093E00CD03197D9F708953197F1F70895BF
:10007000689462F80895E89462F80895EF93FF9306
:10008000EE27E82BE92B31F0EAEFF0E03197F1F7BA
:0A0090000197D1F7FF91EF91089559
:00000001FF
